:020000040000FA
:100000008A01B301B2011D2AB6000308B7008312AA
:100010000B11B330B11B2C3E8100B11F13280830E7
:10002000A706A71D1628900A2C3093072708061943
:10003000103A1039031D2028271DA70A21211C2949
:100040006400A70614088207112936293B293E2996
:1000500046292121A713271DA717BF22820711298F
:1000600094031929160E0F3982070F340734073409
:1000700003340334013401340034003401340134D6
:1000800003340334073407340F341D1A4A290F3060
:100090001D0582072C2A142A262B262B262B262BDD
:1000A0000C2B0C2B262B262B102B0E2B262B262B2A
:1000B000262B122B1B083906031D67281C082A064D
:1000C000031D67281D08C039803A031990281B08B2
:1000D000031D3F2AF0301C05703A031D3F2A0630ED
:1000E00095003114BC01EC22B11E3F2A1E089F006E
:1000F0001D089E001C089D009918A828E2282818B1
:100100001D2A31111C081B04031990281C082906FC
:10011000031D5A281B083806031D5A28B11831152B
:10012000BC0106309500EC229D08031D3110B4017E
:10013000B40A9D0E1D0C9D0E0739820745286A2BB7
:100140007C2B7C2BB42BC42B3E2AB40A1D1AE2282C
:10015000B40A3119262B1E08AB001D080339C5232C
:1001600089001F089E009D0C1D0C03398207262B59
:10017000C128C628BB28B11E262B1E085F21122BC2
:1001800089005A211E060319122B262B1E08073937
:10019000AE00AE0AAD010314AD0DAE0BCC285A2152
:1001A000AE001E1ADA282D082E059E192D060319F9
:1001B000122B262BB11E262B2D082E049E1D2D063C
:1001C0005F21122B1D0807398207ED28ED28ED2845
:1001D000ED28F428F628C028C0283207311C143E28
:1001E000AB003308C5230D2913300D299E03AB0145
:1001F00003109E0DAB0D9E0DAB0D9D1D04291E0819
:10020000B2002B08B300122B1E083206031D262B4A
:100210002B083306031D262B122B89009D1DC12898
:10022000BB289401B117123099009A011B30840049
:10023000940AF830A705A70A37088300B60E360ED1
:1002400009002818080012081302031C0800930074
:100250008D0A8D0A0F080D02031C32290511033087
:10026000860408003F08860505150800271911298E
:10027000990B192918292719940A1929271D1129B9
:10028000B1132A308102FE3098001829A70A940A77
:1002900021211C29B40A0E301D05023A031D262B0C
:1002A0009E131D1C9E170D3089001E085F21262BF2
:1002B00083128900831608148312080808008B1320
:1002C00064008312880006300906FE3903197B2971
:1002D0008316081555308900AA30890088148818BB
:1002E0006F29081183128B177B2901309100C030D0
:1002F000B1008030A70008305821AF00AF0DAF0D1E
:1003000083302F04920013305821BA00BA1E93296B
:100310000C305821AA00A9000B305821E739C03809
:10032000B900B8009A29B901B801003058217F39C5
:10033000AA00A900B1100D305821AF003112AF1B37
:1003400031167F3903190800A900B801B11408005B
:10035000133089003A085F210800AC000830AD0076
:100360002C08AC01AB0C0318AC07AC0CAD0BB229DC
:10037000AB0C08000C08031DBF298F0108003A1EB2
:10038000D229AB001B30AD212430AC072C085821FA
:10039000AE002C035821AF002E02AD212C082F07F0
:1003A0008F000800B00104305821FE390319FF30D6
:1003B000AB000310AB0C01305821AE000310AE0CA3
:1003C0002E08AB070C08AD212E082C020318EA29D1
:1003D000B00A003CAB0080300C020318F229003C4C
:1003E000B00AB017AD21AB0D2C0D3018003CAF009A
:1003F0000C08AB00003CAD2105305821FE39031933
:100400008030AB000310AB0C2C08AD21AB0DAC0D54
:10041000AB0D2C0DAF07AF1B102A2F0D033ED029BB
:100420000030B01FFF30D0290D30890003015F215B
:10043000BA01A8210301890A5F218B13A801031ABD
:10044000262A13305821BA003A192814BB17A530B0
:100450003D0603193D2ABD0675218B133F309700D9
:100460008C018E018F018D01900185018601FC3088
:10047000BF0006128612BC01BB01552394019901ED
:100480001B3084009A019F01A00127138B160B11CA
:100490008B179422271B7F280A3058210319492AD9
:1004A0003C02031C492AB02B960A0319BC0A1830D7
:1004B000970540301605833897049712171F971633
:1004C00032201605031D17150630160503191710DF
:1004D0007830160503199710BE0B722A97130F0C6C
:1004E000FF3CBE00AF010530B0000130AD002D086B
:1004F0003B050319852A3008213C58211705031DA7
:10050000852A30081C3C5821AF040310AD0DB00BF8
:10051000772A0030AF062F080506033985062F0815
:10052000060670398606080028180034503010027C
:10053000031CBE2A90005422950B9F2A3110910B68
:10054000BE2A0C080E020319BD2A031CAD2A8C0A10
:100550000230582191001030B22A8C030330582108
:10056000910011305821AB007F39AB1B003C910743
:10057000031DBC2A0E088C00BA21910A0034270DF5
:10058000A71ECF2AA712031CCF2A31179A08031DD2
:10059000003404309902031C0034990A2717980D7F
:1005A00003180134A716271B003418089A06311FB8
:1005B000E22A3113C039C03A0319E12A9B01840AA7
:1005C000990A18088000840A990A0730190203184A
:1005D0000034980198090134B1161B082106031D47
:1005E000B112A1061C082206031DB112A2061D08A5
:1005F0002306031DB112A3061E082406031DB11213
:10060000A4061F082506031DB112A506200826060C
:10061000031DB112A6060800A821122BBA160C2B36
:10062000BA120C2B311C262B8B131030AD00061682
:1006300086168610061405156400AE01AE0B1E2B3F
:10064000AD0B1C2B0610061286123E2A34089902A6
:100650000319402A031C3E2A1E089D001F089E0005
:1006600020089F00B40B2C2B9728311D3A2B311AF0
:100670002B063C2B3A182B062B05031D442B3F1051
:100680001716BF1497110800BF1097153F141712C3
:1006900008000F305821311D0330FF3ABB05FF3AE7
:1006A0001D1E0301BB041D1208008316CB30810000
:1006B00028185F2B0030850084308600682B0430BA
:1006C0008500873086008312003085003030860038
:1006D000831208001D083F3A031D262BB40A803000
:1006E000AB001E0835231E0DFE390319B12BFE3E4B
:1006F0000319B02BFE3EAA2BB1112030AB001D0810
:100700003523BA1C49231F309D051D080F390319D5
:10071000B12BFF3E0319B02B03109D0D9D1A1D1424
:100720009D1235081D020318972BB115023EFF3E9E
:10073000B0001D08B500FC3EAB009730AD21AC0EFB
:100740002B0E2C060F392C06B008031DAA2BB11D49
:10075000F63E053E013E8E00BB1B8C00BB13B22B48
:100760008C018E01BA21262BBA1849239D0D9D0DAF
:100770003B089D060E305821AB00AB0C2B0C3C39CE
:10078000311D3C301D05BB06262B0339031DFF34EC
:100790000B302B020318CE2B0B3E080010302B021F
:1007A000031CFF34FD3E0318D72B0E3E0800143007
:1007B0002B02031CFF34FB3E0318E02B133E080002
:1007C0001C302B02031CFF34F73E0318E92B1C3EA0
:1007D000080030302B02031CFF34FB3E0318F22BC1
:1007E000213E080040302B02031CFF34E13E031879
:0607F000FF34403E08004A
:084000000000000000000100B7
:02400E00F63F7B
:104200000300070000000000010001006900A50094
:10421000000000000000000000000000000000009E
:10422000000000000100000000000000000010007D
:10423000200040000100020014000A00800000007D
:0242400000007C
:0C4244008000010006000C0010001400B7
:1042500018001C00200024002A00300036003C001A
:1042600044004C0054005C00660070007C00880034
:104270009800A800BC00D000E600FC00FF00800011
:00000001FF
